:020000040000FA
:100000008A150A16612DFF3F212E0800FF3FFF3F92
:10001000FF3FFF3FFF3FFF3FFF3FFF3FFF3FFF3FF0
:100020008A150A1600208A110A123126F012F212DD
:10003000F213E101E2018611701183120313F8013A
:10004000F901FA01FB01FC01FD01FE01FF01203075
:1000500084000021A000243020020319B8293C307C
:100060002002031D2928840AD5010230DE00002168
:10007000D507D6208000840ADE0B37282208D4005A
:10008000210ED40406305402DE000021D507D6200C
:100090008000840ADE0B45280230DE000021D620D5
:1000A0008000840ADE0B4E280021DD003E305D0218
:1000B000031D812884030008DD008403000EDD0495
:1000C00055085D02031D8A2883132430840000082C
:1000D000D6008403000ED604D60803197E284E30BD
:1000E000560203187E2806118615903056070730F1
:1000F0000318013E8A00560890271B280030E000B4
:1001000099280130E00099280230E0009928033056
:10011000E00099280430E00099280530E000992893
:100120000630E00099280730E00099280830E00008
:1001300099280A30D4000030D6008317103084008C
:1001400060088000061570154F211B2841346C345F
:100150006C34203459346F34753472342034423462
:10016000613473346534203441347234653420345E
:10017000423465346C346F346E3467342034543414
:100180006F34203455347334FF3FFF3FFF3FFF3F50
:10019000F6308100D428EC308100D428D83081009A
:1001A000D4283D308100D4280B110800F700F60058
:1001B0000F30F605473077020318E4284130770204
:1001C000031CE4280930F60776080800CD00CE00AD
:1001D000F030CE054E0EF220CE000F304D05F2204D
:1001E000CD000800F6000A307602031CFA283730EA
:1001F0007607FC28303076070800F01C11293629D4
:10020000F01C03291F2983120313F01A0F29061467
:100210008316891B0C290929831206100808061069
:100220000800F01A1E2983128C1388000614831606
:10023000091B182983128C1F1B2906100800831222
:1002400003138C1A272986128C1A272924291A08A5
:10025000312918192F2998182F290301312918122B
:1002600018168616CF01CF0B33290800D3000C1EB9
:100270003729530899008316981C3C29402983127A
:100280008312080004305402D1008313213084000B
:10029000D5010008D507840AD10B4929080083132A
:1002A000203084005B308000840A5408E6204E0829
:1002B0008000840A4D088000840A5608E6204E0813
:1002C0008000840A4D088000840A701D842908304B
:1002D0005402D1000310D10C2530D2008317103006
:1002E000F7008317770884000008E620831352087C
:1002F00084004E088000D20A840A4D088000D20A89
:100300008317F70AD10B7129422103305402F600FA
:100310002030760784005508E6204E088000840AC5
:100320004D088000840A5D3080005408D10083139A
:10033000203084000008FD20840AD10B9A2908008F
:100340008312031386168316403099008312181205
:100350001A081A0818160800831203138616831643
:1003600015309900831218121A081A081816080076
:100370000530DE002130840000218000840ADE0B7D
:10038000BC29DD000D305D02031D7E283030FD20CC
:100390003230FD201B280E30D4000130D6008A11E7
:1003A0000A1600208A110A1270154F210800123017
:1003B000D4000230D600422670154F2108000E30BE
:1003C000D4000430D60070150230DA008A150A16FF
:1003D00007208A110A12711CF0291925E0009E25B8
:1003E00070154F2108000830D4000530D600831363
:1003F0002608DD00250EDD04DD080319002A022A87
:100400005827032A51274F2108000830D40006300E
:10041000D6002608E300250EE3042808E400270E92
:10042000E4042908E5002A0EE5044F2108000A30FB
:10043000D4000730D6008A110A160C208A110A123D
:1004400070154F2108000A30D4000830D600A926C4
:1004500070154F2108000830D4000930D600260856
:10046000E200250EE2044F2108000830D4000A30D3
:10047000D6002608DD00250EDD04F212DD08031982
:10048000422AF2164F2108000830D4000B30D60063
:100490002608DD00250EDD04DD080319502A572A41
:1004A0008A110A16D2218A110A12F2135D2A8A11C0
:1004B0000A16D2218A110A12F2174F2108000830B9
:1004C000D4000C30D6002608DD00250EDD047213A2
:1004D000DD08031D6C2A72170B30DA008A150A1624
:1004E00007208A110A124F21080008000800831211
:1004F0000313F016061008000830D4001230D6009E
:100500004F2108000830D4001B30D6008A110A168B
:10051000AA218A110A120430DA004B25080008309B
:10052000D4001E30D6008A110A16AA218A110A1296
:100530000330DA00282508000830D4002330D60024
:100540008A110A16B0218A110A121C30DA002825F5
:1005500008000830D4002430D6008A110A16B021D1
:100560008A110A121D30DA004B2508000830D40029
:100570002530D6004F218A110A16D2218A110A127B
:1005800008000830D4002630D6008A110A168821C7
:100590008A110A124F2108000830D4002730D600F3
:1005A0008A110A168B218A110A124F21080008307D
:1005B000D4002830D6008A110A16D2218A110A12D4
:1005C0004F210B2D0830D4002930D6008A110A168D
:1005D00079218A110A124F2108000830D4002A30EC
:1005E000D60083132608DF00250EDF048A110A16C1
:1005F000B3218A110A124F2108000830D4002B3091
:10060000D6002608DD00250EDD0400305D0203194A
:10061000142B01305D020319282B02305D020319EF
:10062000122B3B2B17273B2B17271D2604271D2694
:10063000492787193B2B4127871587114927D12047
:1006400087193B2B0B1D202B0730E0009E253B2BF1
:1006500017271D2604274127871587114927193099
:10066000DA008A150A1607208A110A12711C3B2B20
:100670001925E0009E254F2108000A30D4002C30B7
:10068000D600F2184B2B7219492B0030D6000330DC
:10069000592B0230592B4927871D572B5030DE002C
:1006A000871D572BDE03031D502B0030592B0130C3
:1006B000592BDD00831710308400831203135D086B
:1006C000800070154F21080017271D2604270830C9
:1006D000D4002D30D6004F2108000830D4002E3031
:1006E000D6008711412787113827071E7D2B8A15D1
:1006F0000A1698228A110A12742B871519261926B0
:10070000871149274F2108000830D4002F30D60028
:100710001A30DA00092E0830D4003030D6001930F3
:10072000DA00092E0830D4003130D600AA258A110B
:100730000A16D2218A110A12B12508000830D40005
:100740003230D600C6258A110A16D2218A110A1221
:10075000D22508000830D4003330D6002608DD004A
:10076000250EDD0400305D02031DB82B1727C72BB3
:1007700001305D02031DBE2B0427C72B02305D0232
:10078000031DC42BF126C72B0630E0009E254F2108
:1007900008000A30D4003430D600831710308400AB
:1007A000B426831203131E088312031780008312DA
:1007B000031370154F2108000A30D4003530D600DD
:1007C000831710308400F126B026172783120313F5
:1007D0001E088312031780008312031370154F2124
:1007E00008000A30D4003730D60083171030840058
:1007F000B826831203131E08831203178000831286
:10080000031370154F2108000830D4003930D6008A
:10081000C6258A150A16EB208A110A12F11C132C20
:1008200070160730E000D22508000830D4003B30B5
:10083000D6002508DD0001305D020319232C0630A7
:10084000E0009E252D2C8A110A16A7218A110A1272
:10085000711D2D2C0730E0009E254F210800083027
:10086000D4003C30D600F801F901FA01FB01FC018B
:10087000FD01FE01FF018A150A16EB208A110A12FA
:100880004927871D402C472C0730E0009E254F212B
:1008900008001030D4003D30D60070150D30DA005D
:1008A000092E0830D4003E30D600AA258A110A1637
:1008B000D2218A110A12B1258A110A1208000830C1
:1008C000D4003F30D600C6258A110A16D2218A11DB
:1008D0000A12D22508000830D4004030D600AA25DC
:1008E0008A110A1631218A110A12B125080008302E
:1008F000D4004130D600C6258A110A1692208A11EA
:100900000A12D22508000830D4004230D6007C25D7
:100910008A110A16A7218A110A124F2108000830ED
:10092000D4004330D600C6258A110A1612208A1137
:100930000A12D22508000830D4004430D600C6255B
:100940008A110A1634208A110A12D22508000830AA
:10095000D4004530D600C6258A110A1671208A11A6
:100960000A12D22508000830D4004630D600C62529
:100970008A110A164F208A110A12D225080008305F
:10098000D4004730D600AA258A110A16AE208A1153
:100990000A12B1258A110A1208000830D400483022
:1009A000D600AA258A110A16D3208A110A12B12567
:1009B00008000830D4004930D600AA258A110A164A
:1009C00012218A110A12B12508000830D4004A30D9
:1009D000D600AA258A110A16F3208A110A12B12517
:1009E00008000830D4004B30D6002608E100250E60
:1009F000E1044F2108000830D4004C30D6004F21CC
:100A00001D26A02108000830D4004D30D6004F210B
:100A10001D26AC2108000030E0000A30D400003070
:100A2000D6008317103084006008800070154F21B5
:100A30000800F11D1D2D0930272D711E212D1030AC
:100A4000272D711F252D1130272D0830272D080047
:100A50007C258A150A1607208A110A12711C342D6A
:100A60000730E0009E25492D4F2115267B30FD20C3
:100A70001526D5018A150A16BB218A110A125508B6
:100A8000E6204E08FD204D08FD2015267D30FD2076
:100A900015264F2108007C258A150A1607208A1181
:100AA0000A12711C572D0730E0009E257A2D4F2128
:100AB00000217B3C0319602D0130E0009E257A2D3A
:100AC000D5018A150A16D2218A110A120021D620D0
:100AD000DD00DD0E0021D6205D0455020319732DC3
:100AE0000430E000701600217D3C03197A2D01309E
:100AF000E0009E254F21080083132C08F8002B0EE0
:100B0000F8042A08F900290EF9042808FA00270E2B
:100B1000FA042608FB00250EFB043408FC00330E03
:100B2000FC043208FD00310EFD043008FE002F0EDB
:100B3000FE042E08FF002D0EFF0408000A30D4002A
:100B40000030D600701583171030840060088000D4
:100B5000061508007C254F2115267B30FD20D50188
:100B600008005508E6204E08FD204D08FD207D3088
:100B7000FD20C42D0A30D4000030D6007015831734
:100B800010308400600880004F21080070127C251E
:100B90004F2100217B3C0319D02D0130E00070165D
:100BA000D50108000021D620DD00DD0E0021D62071
:100BB0005D0455020319DF2D0430E000701600219A
:100BC0007D3C0319E62D0130E000701603138312FB
:100BD000701EF42D0A30D4000030D6007015831733
:100BE00010308400600880004F210800E6204E0885
:100BF000D507FD204D08D507FD2008000021D507A9
:100C0000D620CE00CE0E0021D507D620CE044E0829
:100C100008008A150A1607208A110A12711C132E61
:100C20000730E0009E254F210800C8200B1D162E1E
:100C30000800CE200B1D1A2E0800D1200B1D1E2EE1
:100C40000800F300030E8301F5000A08F4008A018E
:100C50000B18E12274088A00750E8300F30E730EE0
:100C600009008316D0308700A0000514851485156F
:100C700004309F00831280309F0017278030E800E7
:100C8000C426080086157208E7002327831203177D
:100C9000103084006126840A6D26840A7926840A2D
:100CA0008226840A8F26031383126708F2007218C3
:100CB000F126F218042772191727F2192327861133
:100CC000080003138312B42633301E02031C9D2E2A
:100CD0009A301E020318A12EA52E03138312B826E4
:100CE00047081E02031C9D2E49081E020318A12E50
:100CF000A52E031383121727B026A4081E0203187B
:100D0000A12EA52E031383120427B42633301E020E
:100D1000031C9D2E9A301E020318A12EA52E03132C
:100D20008312F126B026172747081E02031C9D2EAA
:100D300049081E020318A12EA52E8317013080003A
:100D4000080083178030800008008317003080007F
:100D500008008317103084000030831780000800DB
:100D60009F121F129F11BC2E9F121F129F15BC2E87
:100D70009F121F169F15BC2E5F271F145F271F157C
:100D80001F19C02E1F100800031383128610113084
:100D9000E600D0266808E600D026861463270800FF
:100DA0000830D000E60D031CD72E8617D82E8613E8
:100DB0000000000000000000061700000000000016
:100DC00000000613D00BD22E0800861406178617D3
:100DD0000800861406178613080086140617861363
:100DE00008000708EC006C15EC146C106C08870008
:100DF0007214F2107211F2118A110A12D1208A11A2
:100E00000A120B1D012F08000708EC006C15EC10EE
:100E10006C146C0887007210F2147211F2118A11AE
:100E20000A12D1208A110A120B1D142F080007087C
:100E3000EC006C11EC146C146C0887007210F2104A
:100E40007215F21108000708EC006C15EC146C1414
:100E50006C0887007210F2107211F21508009412DB
:100E600083162016A012200887008312851608001A
:100E7000941283162016A01620088700831285126C
:100E8000080094128316A01120088700831205150C
:100E9000080094128316A0152008870083120511FC
:100EA0000800051281010B110B1D542F721208004E
:100EB000051681010B110B1D5B2F72160800CF0167
:100EC000CF0B602F0800CE200B1D642F08000030D0
:100ED000EA006A08E800C426F126B0261727480869
:100EE0001E020318782FEA0F692F0030E800C4268D
:100EF0000800FF3FFF3FFF3FFF3FFF3FFF3FFF3F38
:100F0000FF3FFF3FFF3FFF3FFF3FFF3FFF3FFF3FF1
:100F1000FF3FFF3FFF3FFF3FFF3FFF3FFF3FFF3FE1
:100F200082070000CB29D7290B2DDF29F329052AB9
:100F3000172A232A2B2A352A442A5F2A0B2D752AA1
:100F4000762A0B2D772A7C2A0B2D0B2D0B2D0B2DA2
:100F50000B2D0B2D0B2D0B2D822A0B2D0B2D8F2ADC
:100F60000B2D0B2D0B2D0B2D9C2AA92AB62AC12A3D
:100F7000CC2AD72AE22AED2AFD2A3D2B642B6D2BA1
:100F8000842B8B2B922B9E2BAA2BC92BDC2B0B2D6E
:100F9000F12B0B2D042C0B2D152C2F2C492C512C07
:100FA0005F2C6B2C772C832C8F2C9B2CA72CB32C99
:100FB000BF2CCD2CD92CE52CF12CFB2C032D0B2D8B
:100FC0000B2D0800FF3FFF3FFF3FFF3FFF3FFF3F6D
:100FD000FF3FFF3FFF3FFF3FFF3FFF3FFF3FFF3F21
:100FE000FF3FFF3FFF3FFF3FFF3FFF3FFF3FFF3F11
:100FF000FF3FFF3FFF3FFF3FFF3FFF3FFF3FFF3F01
:1010000008308A005F088207003400340034322D33
:101010004E2D642DAA2DAB2DAC2DAD2DD22DD92D5D
:1010200008308A005F088207003400340034E32D62
:10103000012E5B2E5C2EE62EE72EE82ED22DEA2E18
:1010400008308A005F088207003400340034322DF3
:101050005D2D642D5D2D642D5D2DCA2D5D2DFF341C
:1010600008308A005F088207003400340034322DD3
:10107000562D642D562D642D562DC02D562DFF3422
:1010800008308A005F0882070034003400340134DD
:10109000083401340434013404340134023401349A
:1010A0000234023408308A005F08820700340034BA
:1010B0000034013404340134043401340434013480
:1010C00001340134023402342E2908308A005F08CA
:1010D0008207003400340034F12A112B362B432BC5
:1010E000902B912B922B932BB72B08308A005F0803
:1010F0008207003400340034CB2BD12BD22BD32BDE
:10110000D42BD52BDB2BDC2BE32B08308A005F089C
:101110008207003400340034D92CEE2C062D0D2D1E
:101120002C2D2D2D2E2D2F2D312D08308A005F08CE
:101130008207003400340034592C7C2CA12CAE2CB6
:10114000AF2CB02CB12CB22CC62C08308A005F0812
:101150008207003400340034EE2B0A2C1C2C1D2C8A
:10116000352C362C372C452C462CFF3FFF3FFF3FBC
:10117000FF3FFF3FFF3FFF3FFF3FFF3FFF3FFF3F7F
:10118000FF3FFF3FFF3FFF3FFF3FFF3FFF3FFF3F6F
:10119000FF3FFF3FFF3FFF3FFF3FFF3FFF3FFF3F5F
:1011A000FF3FFF3FFF3FFF3FFF3FFF3FFF3FFF3F4F
:1011B000FF3FFF3FFF3FFF3FFF3FFF3FFF3FFF3F3F
:1011C000FF3FFF3FFF3FFF3FFF3FFF3FFF3FFF3F2F
:1011D000FF3FFF3FFF3FFF3FFF3FFF3FFF3FFF3F1F
:1011E000FF3FFF3FFF3FFF3FFF3FFF3FFF3FFF3F0F
:1011F000FF3FFF3FFF3FFF3FFF3FFF3FFF3FFF3FFF
:1012000002293322BD08031D0829BC0803190E2931
:101210000130BC0203180129BD02012908000D227A
:101220005F21080020225F2108000D225F210800B5
:101230008A110A168E218A150A12871287118A11BD
:101240000A12F1268A150A127908BD007808BC0036
:1012500021303D0603192D29002108008A110A16A4
:101260008E218A150A12871287118A110A12F12615
:101270008A150A127908BD007808BC0008008A1196
:101280000A168E218A150A12871287118A110A12EC
:10129000F1268A150A12C121A121BD017808BC00DE
:1012A000002108008A110A168E218A150A12871257
:1012B00087118A110A1217278A150A120800BA0123
:1012C000BB018A110A1695218A150A128715871102
:1012D0000830D000871587110310871A0314BA0C41
:1012E000D00B6A290630D000871587110310871AA2
:1012F0000314BB0CD00B7429BB0CBB0C87158711D6
:101300008A110A168E218A150A120800871287157B
:1013100087110830D0008716B80C031C8712871578
:101320008711D00B8B290630D0008716B90C031C0F
:10133000871287158711D00B95298712871587117A
:1013400008003908C6003808C500FF30B900B800E9
:1013500086214608B9004508B80008000130F700AA
:10136000B7290230F700B7290430F700B7298A11EE
:101370000A12CE208A150A120B1DBC29F70BB729B9
:101380000800871287158711871287158711871222
:10139000871587118712871587118712871587117F
:1013A00087128715871108008716871587118712FE
:1013B000871587118712871587118712871587115F
:1013C00087128715871187128715871108008712E2
:1013D000871587118716871587118712871587113B
:1013E000871287158711871287158711871287152E
:1013F00087110800871687158711871687158711AB
:10140000871287158711871287158711871287150D
:101410008711871287158711080087128715871192
:1014200087128715871187168715871187128715E9
:101430008711871287158711871287158711080072
:1014400087168715871187128715871187168715C5
:1014500087118712871587118712871587118712C1
:10146000871587110800871287158711871687153A
:10147000871187168715871187128715871187129D
:10148000871587118712871587110800871687151A
:101490008711871687158711871687158711871279
:1014A000871587118712871587118712871587116E
:1014B00008008712871587118712871587118712F1
:1014C000871587118716871587118712871587114A
:1014D00087128715871108008716871587118712CD
:1014E000871587118712871587118716871587112A
:1014F00087128715871187128715871108008712B1
:101500008715871187168715871187128715871109
:1015100087168715871187128715871187128715F8
:101520008711080087168715871187168715871179
:1015300087128715871187168715871187128715D8
:101540008711871287158711080087128715871161
:1015500087168715871187168715871187168715B0
:101560008711871287158711871287158711080041
:10157000871287158711871287158711871287159C
:101580008711871687158711871687158711871288
:101590008715871108008716871587118716871505
:1015A0008711871687158711871287158711871668
:1015B00087158711871287158711080087168715E9
:1015C0008711871687158711871687158711871644
:1015D0008715871187168715871187128715871139
:1015E00008008A110A166D21B8006D21B9008A150C
:1015F0000A12E72186210130610203190C2B8A119E
:101600000A12B4268A150A1276301E02031C0C2B0D
:10161000B822B421C001102B5922B421B421C00139
:1016200008008A110A166D21B8006D21B9008A15CB
:101630000A12E7218621C00A4A084006031D352BFD
:10164000E108031D312B8A110A12B4268A150A12E9
:1016500076301E02031C312BB822AE21CB22C001F2
:10166000352B5922B421B421C00108008A110A1671
:101670006D21B8006D21B9008A150A12E721862173
:101680005922B4210800E10803197C2B472B522171
:10169000AE21F901F8011821FF30B800B900E721A7
:1016A00086215922B121B121CB220830C6008A11EE
:1016B0000A166D21B8006D21B9008A150A12E721BA
:1016C00086210330C50033228A110A166D21B80025
:1016D0006D21B9008A150A12E7218621C50B632BFB
:1016E000B822B121B121CB223322C60B572BFF01E7
:1016F000FE01FD01FC018F2B8A110A166D21B80035
:101700006D21B9008A150A12E7218621C00A04302A
:101710004006031D8F2BB822B121CB22C001080047
:10172000362B432B362B8A110A166D21B8006D21FA
:10173000B9008A150A12E7218621C00A8A110A1601
:1017400050218A150A128A150A1233228A150A12A2
:101750008A110A166D21B8006D21B9008A150A1286
:10176000E72186215922AE21A522C00108008A1155
:101770000A166D21B8006D21B9008A150A12E721F9
:101780008621C00AB822B121A5228A110A12C820D6
:101790008A150A120800E72186215922B421B421B2
:1017A0000800CB2BCB2BCB2BCB2BE721862159222F
:1017B000B121CB220800CB2BE721862159225922C7
:1017C000AE21A5220800E7218621B822B121A52259
:1017D0008A110A12C8208A150A1208008A110A16EC
:1017E0006D21B8006D21B9008A150A12E721862102
:1017F000E108031D072C8A110A12B4268A150A1261
:1018000076301E02031C072CB822B421092C592261
:10181000B42108008A110A166D21B8006D21B900A3
:101820008A150A12E7218621B822AE21CB221B2C71
:101830005922B421B42108000A2CFF30B800B900A5
:10184000E72186215922B121B121CB228A110A1622
:101850006D21B8006D21B9008A150A12E721862191
:10186000B822B121B121CB2208000A2C1D2C8A11EB
:101870000A166D21B8006D21B9008A150A12E721F8
:1018800086215922B421B42108000A2C8A110A1693
:101890006D21B8006D21B9008A150A12E721862151
:1018A000B822B121A5228A110A12C8208A150A126B
:1018B00008008A110A166D21B8006D21B9008A1539
:1018C0000A12E7218621C00A4B084006031D7B2C23
:1018D000E108031D782C8A110A12B4268A150A120F
:1018E00076301E02031C782CB822B421C0017B2C58
:1018F0005922B421C00108008A110A166D21B800CE
:101900006D21B9008A150A12E7218621C00A4B0809
:101910004006031DA02CE108031D9C2C8A110A120D
:10192000B4268A150A1273301E02031C9C2CB8229E
:10193000AE21CB22C001A02C5922B421B421C00178
:1019400008008A110A166D21B8006D21B9008A15A8
:101950000A12E72186215922B4210800432BA12C29
:10196000AE2CA12C8A110A166D21B8006D21B90088
:101970008A150A12E7218621C00A4B084006031D7A
:10198000C52C5922AE21A522C00108008A110A16D1
:101990006D21B8006D21B9008A150A12E721862150
:1019A000B822B121A5228A110A12C8208A150A126A
:1019B0000800FA218621E108031DEA2C8A110A1287
:1019C000B4268A150A1276301E02031CEA2CB822AD
:1019D000B421EC2C5922B42133220800FA218621AB
:1019E000E108031D012D8A110A12B4268A150A1274
:1019F00076301E02031C012DB822B421B421CB2263
:101A0000042D5922B421B42133220800FA21862161
:101A10005922B421B42133220800FA218621E10899
:101A2000031D202D8A110A12B4268A150A12763057
:101A30001E02031C202DB822B421B421CB222A2D52
:101A40005922B121B121B121B121CB22B822B1213A
:101A5000B121CB2233220800062D0D2D062D003496
:101A60000800FF342030F9000730F8003F210F2133
:101A7000BB123B133B08B9003A08B800CB235221F4
:101A80002030F9000730F8003F21D42146225922A6
:101A9000B421B421D421462252210800F801F901D1
:101AA0003F21DE22B421B421522108006C22B4214E
:101AB000B4215922B421B42108009222B421B421C6
:101AC0005922B421B421080018210430C500FF3088
:101AD000C6003322C60B692DC50B672D3322332276
:101AE000332215213A08C2003B08C30052213F218E
:101AF0000F2143133B1A4317C313BB1AC317C1214A
:101B0000A1216C22B421B4219222B421B42152210A
:101B100018210430C500FF30C6003322C60B8D2DBE
:101B2000C50B8B2D3322332233224208B8004308E1
:101B3000B9003E2352213F210F213B12431B3B168C
:101B4000BB12C31BBB163A08B8003B08B900D2232E
:101B5000522108004E2D642D4E2D2030F900073003
:101B6000F8003F21E721A1216C22B421B421B42146
:101B7000B4219222B421B421B421B421522108000D
:101B80001821E721A1216C22B421B421B421B42170
:101B90005221080018219222B421B421B421B42189
:101BA00052210800F801F9013F216C22B421522191
:101BB00008003F21C121A1216C22B421B121B4210F
:101BC000B12152210800F801F90118216408C4006C
:101BD0006508C500EC2D3322FF30B800B900E721BD
:101BE00086215922B421C408031DF92DC508031903
:101BF000FF2D0130C5020318EB2DC402EB2D52213D
:101C000008000330F6006308C4006408C5006508D6
:101C1000C6000310C40CC50CC60CF60B092EF90146
:101C2000F80118210830F600FF30B800B900E721AC
:101C30008621F60B1C2E1E2E3322142E5922B4217F
:101C4000B421C408031D2A2EC508031D2A2EC60868
:101C50000319352E0130C6020318332EC5020318AE
:101C6000332EC402332E3322122EC1210430C6007B
:101C7000FF30B800B900E72186215922B421B421F0
:101C8000C60B432E452E3322382E3322FF30B800A8
:101C9000B900E72186215922B421B421332233220D
:101CA0003322FF30B800B900E72186215922B42140
:101CB000B42152210800642D8026C7266026080022
:101CC000F801F9013F21FF30B800B900E721862172
:101CD0005922B121B121CB220230C5000430C60007
:101CE0003322FF30B800B900E7218621C60B702EE1
:101CF000B822B121B121CB22C50B6E2E5221080092
:101D00000530F6006308C4006408C5006508C60015
:101D10000310C40CC50CC60CF60B882EF901F80193
:101D20001821FF30B800B900E72186212030CC000F
:101D30000430F6005922B121CB22A12E0430F60046
:101D40003322FF30B800B900E7218621CC03F60B1F
:101D5000A02EB822B121B121CB22CC080319B12E7B
:101D60009E2EC408031DBA2EC508031DBA2EC60830
:101D70000319E42E0130C6020318C32EC50203184E
:101D8000C32EC402C32E3322962E52210800B12145
:101D9000B121F901F8012E21FF30B800B900FA2174
:101DA0008621C6015922B121B121CB22FF30B800D2
:101DB000B900FA218621B822B121B121B121B12186
:101DC000CB223322C60BD22E52210800642D5C2E6A
:101DD000AD2DD22DFF34FF3FFF3FFF3FFF3FFF3FC1
:101DE000FF3FFF3FFF3FFF3FFF3FFF3FFF3FFF3F03
:101DF000FF3FFF3FFF3FFF3FFF3FFF3FFF3FFF3FF3
:101E0000FF3FFF3FFF3FFF3FFF3FFF3FFF3FFF3FE2
:101E1000FF3FFF3FFF3FFF3FFF3FFF3FFF3FFF3FD2
:1020000083171030840002308000840A073080007B
:10201000840A0030800008008317103084000130EB
:1020200080000800F1128A150A1240208A110A164F
:10203000CA00C0018A150A1218218A110A165021F5
:10204000003A03192E288A150A1265208A110A16E9
:102050008A150A1233228A110A161F288A150A12B3
:1020600052218A110A160800F1128A150A126420F8
:102070008A110A165021003A031949286D21B80027
:102080008A150A1285208A110A16BC0F3A28BD0A41
:102090003A288A150A1252218A110A160800F112EA
:1020A000C0018A150A1252208A110A16CB008A151D
:1020B0000A123F218A110A165021003A03196B288F
:1020C0008A150A1295208A110A168A150A123322D5
:1020D0008A110A165C288A150A1252218A110A16D8
:1020E0000800F1128A150A123F218A110A1650219E
:1020F000003A03198C286D21B8006D21B9008A15AA
:102100000A1275208A110A16BC0ABC0A8A150A121C
:1021100033228A110A1677288A150A1252218A1147
:102120000A160800F112C0018A150A123F218A110D
:102130000A165021003A0319A8288A150A12A52068
:102140008A110A168A150A1233228A110A16992848
:102150008A150A1252218A110A160800F1128A15EC
:102160000A1218218A110A165021003A0319CD28A3
:102170008A150A1215218A110A163A088A110A12BA
:10218000F6253B088A110A12F6258A110A168A15C5
:102190000A1233228A110A16B4288A150A12522109
:1021A0008A110A160800F1128A150A1264208A118F
:1021B0000A165021003A0319ED288A150A12122135
:1021C0008A110A163A0873218A150A1233228A11D3
:1021D0000A16BC0FD928BD0AD9288A150A1252211D
:1021E0008A110A160800F1128A150A123F218A1173
:1021F0000A165021003A03190C298A150A121521D2
:102200008A110A163A0873213B0873218A150A12AB
:1022100033228A110A16F9288A150A1252218A11C4
:102220000A160800F1128A150A123F218A110A16AD
:102230005021003A03192B298A150A120F218A11FD
:102240000A163A0873213B0873218A150A123322B1
:102250008A110A1618298A150A1252218A110A1699
:102260000800F1128A150A123F218A110A1650211C
:10227000003A03194A298A150A1215218A110A16E9
:102280003A0873213B0873218A150A1233228A11F6
:102290000A1637298A150A1252218A110A160800CD
:1022A0008A110A16FF08031D5E29FE08031D5E2918
:1022B000FD08031D5E29FC08031900340130FC02EF
:1022C00003186929FD0203186929FE020318692908
:1022D000FF02FF308A110A1608008A110A12FE2531
:1022E0008A110A1608008A110A12F6258A110A169E
:1022F00008008A110A12B4268A110A1676301E02C4
:10230000031C85298A150A1200288A150A1210282A
:102310008A150A1230288A150A1220288A110A12F0
:102320002F2741278A110A1608008A110A12382716
:102330008A110A1608008A150A1262288A150A12DA
:1023400063288A150A1250288A150A1251288A1100
:102350000A1608000130C10008000230C100080060
:102360000230C1000800831203133830C700C121B6
:10237000C800AF30C9008A110A1267278A110A16ED
:10238000D12911308A005F088207003400340034FC
:102390009C349C349C349C349C349C349C34A234B7
:1023A0009C3408000034FF3FFF3FFF3FFF3FFF3FEB
:1023B000FF3FFF3FFF3FFF3FFF3FFF3FFF3FFF3F2D
:1023C000FF3FFF3FFF3FFF3FFF3FFF3FFF3FFF3F1D
:1023D000FF3FFF3FFF3FFF3FFF3FFF3FFF3FFF3F0D
:1023E000FF3FFF3FFF3FFF3FFF3FFF3FFF3FFF3FFD
:103000000313831600309400831294120800831275
:10301000031301305A0603195A2802305A060319BD
:10302000662803305A0603196D2804305A0603191E
:103030007F2805305A060319912806305A060319CD
:103040009D2807305A060319A92808305A06031983
:10305000B52809305A060319C1280A305A0603193F
:10306000D3280B305A060319E5280C305A060319E9
:10307000EB280D305A06031929290E305A06031978
:10308000632918305A060319702919305A06031992
:103090007D291A305A0603197F291B305A06031955
:1030A00081291C305A06031982291D305A0603193A
:1030B00094290800A621711865281D228317103055
:1030C00084005B088000831203130800A621711896
:1030D0006C280330D700E7210800A62171187E284C
:1030E0008A110A16A121D7008A150A16F1218A1120
:1030F0000A16A421D7008A150A1607220800A6215D
:10310000711890288A110A16A121D7008A150A166B
:10311000F1218A110A16A421D7008A150A1607225E
:103120000800A62171189C288A150A16D700F121DB
:103130008A150A16D70007220800A6217118A828A8
:103140008A150A16D700F1218A150A16D700072218
:103150000800A6217118B4288A150A16D700F12193
:103160008A150A16D70007220800A6217118C02860
:103170008A150A16D700F1218A150A16D7000722E8
:103180000800A6217118D2288A110A169B21D7009F
:103190008A150A16F1218A110A169E21D7008A156E
:1031A0000A1607220800A6217118E4288A110A16B7
:1031B0009B21D7008A150A16F1218A110A169E2131
:1031C000D7008A150A1607220800A621DC01721B07
:1031D000DC0A45220800F110831203137C08DC008E
:1031E0004522F119F1147D08DC004522F119F11492
:1031F0007E08DC004522F119F1147808DC00452234
:10320000F119F1147908DC004522F119F1147A085A
:10321000DC004522F119F11416298A110A12FE2543
:103220008A150A16DC004522F119F114FE08031D67
:103230001F29FD08031D1F29FC0803192829013037
:10324000FC0203180D29FD0203180D29FE020D29A9
:103250000800A621711862298A110A169E21D7003A
:103260008A150A168317103084008001840A8001B1
:10327000840A8001840A8001E721831710308400CA
:10328000840A840A840A0008D900103084000008E7
:10329000840A840A840A800010308400590880005F
:1032A000831710308400840A840A0008D900103083
:1032B0008400840A0008840A800010308400840A94
:1032C000590880000800A62171186F297808DC00D1
:1032D00045227908DC0045227A08DC0045220800F6
:1032E000A62171187C297808DC0045227C08DC00C6
:1032F00045227D08DC0045220800A6210800A62101
:1033000008000800A6217118D2288A110A16D221B5
:10331000D7008A150A16F1218A110A16D221D70080
:103320008A150A1607220800A6217118E4288A11B6
:103330000A16D221D7008A150A16F1218A110A1617
:10334000D221D7008A150A160722080071105A08E0
:10335000DC004522711B7114FF30DB001D22711A45
:1033600071145B085C02031D7114DB08031DBA298C
:1033700071141D2208008A110A1650218A150A1696
:10338000003A0319D1294108D7001D22711AD12909
:103390005B088A110A12F6258A150A16D70BC52969
:1033A000BB2908008A110A1650218A150A16003A0C
:1033B0000319E6294108D7008A110A12FE258A1549
:1033C0000A16DC004522D70BDC29D2290800831716
:1033D000103084001D225B088000840AD70BEA2984
:1033E00008007808DC004522D7030319062A79086B
:1033F000DC004522D7030319062A7A08DC0045229F
:10340000D7030319062A7B08DC00452208007C0844
:10341000DC004522D70303191C2A7D08DC00452265
:10342000D70303191C2A7E08DC004522D7030319A1
:103430001C2A7F08DC004522080071126D22F11958
:103440003D2A8A110A1238278A150A169301253057
:10345000940094168C110A30D8008A110A12D120D7
:103460008A150A160B19372A8C1D322A3A2AD80BCC
:103470002D2A3D2A1308DB003E2A711687128A1175
:103480000A122F278A150A1608006D22F1195E2AE2
:1034900071132530940094168C115C0893000A3047
:1034A000D8008A110A12D1208A150A160B195B2A34
:1034B0008C1D562A5F2AD80B512A5E2A71178A1151
:1034C0000A12CB208A150A160B1D642A87128A114C
:1034D0000A122F278A150A160800F1118A110A12FA
:1034E000492787122F278A150A16C6220A30D800C4
:1034F0008A110A12D1208A150A160B19822A871DF1
:103500007D2A852AD80B782A962AD82287160A304F
:10351000D8008A110A12D1208A150A160B19932A8B
:1035200087198E2A972AD80B892A962AF11508001E
:103530008A110A12492738278A150A16DB01071E45
:103540009F2A871DA12A0830D800871DA52A871920
:10355000A72A0310071A0314DB0DD80BA52A871D11
:10356000AF2A8719B12AD8228A110A1241278A154F
:103570000A168715000000000000000087118A115C
:103580000A12492738278A150A1608008A110A12D2
:10359000D1208A150A16DE2A8A110A12CE208A152F
:1035A0000A16DE2A8A110A12CB208A150A16DE2A8A
:1035B0008A110A12C8208A150A16DE2A0B1DDE2A75
:1035C000080000340034000200070000FF3FFF3F06
:1035D000FF3FFF3FFF3FFF3FFF3FFF3FFF3FFF3FFB
:1035E000FF3FFF3FFF3FFF3FFF3FFF3FFF3FFF3FEB
:1035F000FF3FFF3FFF3FFF3FFF3FFF3FFF3FFF3FDB
:10360000FF3FFF3FFF3FFF3FFF3FFF3FFF3FFF3FCA
:1038000083120313FB308605083086041030BE0097
:1038100020308400B02580003C302002031D0A2C9B
:10382000840ABE0B0A2CC3010C30BE002130840078
:103830000008C307840ABE0B182C0A30BE002530CE
:1038400084000008C1258000840ABE0B212C2808B2
:10385000B900270EB9042608B800250EB8042C08B4
:10386000BD002B0EBD042A08BC00290EBC0438087C
:10387000BA003908BB003D08BB07031C402CBA0A3C
:103880003C08BA073C302002031DBB2C3E302F02FF
:10389000031DBB2C2E08F5002D0EF5044308750200
:1038A000031DBE2C1B303A020319592C031C602C3B
:1038B000C12CFF303B020319602C0318C12C602C73
:1038C000003038020319672C03186D2CC12C04300A
:1038D000390203196D2C031CC12CC724B025A0008C
:1038E0007B302002031DBB2CC3013808F4003908CB
:1038F000F300F501F6010430BE0020308400B0254D
:10390000C307C1258000840ABE0B7F2C2308F60064
:10391000220EF6042108F500200EF504FF24000015
:103920000000000000000000000000000000000097
:10393000F30A0319F40A3A087402031D792C3B08B0
:103940007302031D792CB025C125A000B025C12527
:10395000A100200EA10443082102031DBE2CB025A6
:10396000A0007D302002031DBB2C83120313F7300F
:103970008605C724BA2C3130D824692D3430D82498
:10398000692D3630D824692D3730D824692D5B3025
:10399000AA253030AA253830AA253130AA25303062
:1039A000AA254330AA253930AA255D30AA2508006A
:1039B000F500B025A0007D3020020319E42C3E3034
:1039C00020020319E42CD92C5B30AA253030AA251B
:1039D0004130AA253030AA253030AA253030AA251A
:1039E0007508AA253330AA25750AAA255D30AA25AF
:1039F00083120313F730860504308604080003178A
:103A0000831273088D0074088F0075088C00760887
:103A10008E0083168C170C158B1355308D00AA3031
:103A20008D008C14000000000C1103138312080099
:103A30000317831273088D0074088F0083168C1788
:103A40000C140000000083120C08F7000E08F800A8
:103A5000031308008312031386168316403099005F
:103A6000243098008312903098001A081A087010B9
:103A70000800831203138C1A472D81010B11861243
:103A80008C1A472D7018402D0B1D402D492D1A08FA
:103A9000512D18194F2D98184F2D0301512D181223
:103AA00018168616BF01BF0B532DBF010800031364
:103AB0008312061A592D8316981C5C2D83129900C7
:103AC000080083120313D1256625692D2A25E925CF
:103AD00008007010B025F900553079020319812DC6
:103AE000563079020319922D5A3079020319962D16
:103AF000503079020319A42D463079020319A72DFD
:103B0000692D7014F01C852D872D18128A2D8316AF
:103B1000091283128312031306117530AA258A0134
:103B20001030820070147630AA25002C7014831295
:103B3000031306110130AA250130AA250130AA2558
:103B40000330AA257010692D86150611A62D0615BD
:103B50008611A92DF01CAE2D5725AF2D0526080086
:103B6000701CB92DF01CB72DB52D3925C02DF125B0
:103B7000C02DF018BC2DBE2DF010B72DF014B52DB2
:103B80000800FA00F9000F30F90547307A020318EF
:103B9000CF2D41307A02031CCF2D0930F907790867
:103BA0000800031383160B30850010308600903018
:103BB00087001730890004309F008312033087008C
:103BC00000308600103085008316D63081008312C5
:103BD000080003138316173089008312031306109D
:103BE0000800831203133D3081000B110614831665
:103BF000891B002E7018F72D0B1DF72D0301032EC6
:103C000083120610080806100800831203138800A8
:103C100006148316091B0A2E831206100800FF3FA4
:103C2000FF3FFF3FFF3FFF3FFF3FFF3FFF3FFF3FA4
:103C3000FF3FFF3FFF3FFF3FFF3FFF3FFF3FFF3F94
:103C4000FF3FFF3FFF3FFF3FFF3FFF3FFF3FFF3F84
:103C5000FF3FFF3FFF3FFF3FFF3FFF3FFF3FFF3F74
:02400E003A3F37
:08400000FF3FFF3FFF3FFF3FC0
:00000001FF
